:10000000DCEF03F01200FFFF04EF04F01200FFFF2B
:100018000CEF04F01200FFFFFFFFFFFFFFFFFFFFE1
:10002A0000000001776B1E0E716E0401400E096F0D
:10003A00200E0A6F040E0B6F880E086F0401200E43
:10004A000E6F040E0F6F400E0C6F1200550EA76E46
:10005A00AA0EA76EA68212000401226B010E236F5C
:10006A0012000001756B040121510001755D20E247
:10007A0075C000F0016A026A040122510024F36E7D
:10008A0023510120F46E24510220F86EF4CFF7FFB9
:10009A00F3CFF6FF0800F5CF76F000017551EA6A52
:1000AA00250FE96E040EEA2276C0EFFF752BDBD727
:1000BA00F86A1200F00E04012217840EA66E0001DF
:1000CA00756B040121510001755D26E27551EA6ADA
:1000DA00250FE96E040EEA22EFCF03F075C000F097
:1000EA00016A026A040122510024F36E235101209D
:1000FA00F46E24510220F86EF4CFF7FFF3CFF6FF27
:10010A0003C0F5FF0C000F0E000175150F0801E181
:10011A009DDF0001752BD5D71200940EA66E000143
:10012A00756B040121510001755D1EE27551006E67
:10013A00016A060ED89000360136E804FBE1026A2D
:10014A0001BE0268040122510024F36E23510120EA
:10015A00F46E24510220F86EF4CFF7FFF3CFF6FFC6
:10016A0075DF0001752BDDD7F86A1200A66A000157
:10017A00756B040121510001755D10E204012251E1
:10018A0000017525A96EA6807551EA6A250FE96EE8
:10019A00040EEA22A8CFEFFF752BEBD7120000015D
:1001AA00756B040121510001755D15E204012251AC
:1001BA0000017525A96E7551EA6A250FE96E040ECC
:1001CA00EA22EF50A86E040EA66E40DFA6B2FED752
:1001DA000001752BE6D71200C40EA66E0001756BDE
:1001EA00040121510001755D21E27551EA6A250F6A
:1001FA00E96E040EEA22EFCF03F075C000F0016A3F
:10020A00026A040122510024F36E23510120F46E84
:10021A0024510220F86EF4CFF7FFF3CFF6FF03C0A4
:10022A00F5FF0C0013DF0001752BDAD7F86A12000C
:10023A00060E00017A5D03E36D50020B01E082D0E5
:10024A000001770511E104010CBF0DD00401400E35
:10025A00096F400E040108170401087D880E040185
:10026A0008130001776B6ED0040108BF6BD0000140
:10027A00756B04012051320A45E0CD0A34E0F80AD0
:10028A002DE0020A26E0010A1FE0070A18E0010A27
:10029A0011E0030A0AE0070A08E0060A01E041D071
:1002AA00DBDE0001040E756F3DD0DBDE050E0001BA
:1002BA00752738D0FFDE0001010E756F33D02DDFB0
:1002CA000001010E756F2ED051DF050E0001752752
:1002DA0029D065DF0001010E756F24D07DDF000192
:1002EA00010E756F1FD06D960001786B796B000156
:1002FA007807000E795B00017851791101E0F7D790
:10030A00FF0010D0030E0401215D03E10001010E7C
:10031A00756F040E0401215D03E10001010E756F82
:10032A0001D000D00001010E776F000175510AE07B
:10033A0075C00DF4400E04010C1704010C7D880EE3
:10034A0004010C1312006C5002E0000E01D0010EE1
:10035A0000090BE0040100513C0BE842E8420D0899
:10036A0002E1C3EF01F0CCEF01F06C5002E0000EA5
:10037A0001D0010E040901E019D812000001606BD6
:10038A00616B666B676BA1EC02F04EEF02F0020E36
:10039A000001605D09E15CD8040100BD02D0C80E0D
:1003AA0001D0880E006F120093EF02F0040E0001D4
:1003BA007A5D09E112C46EFF6E50000802E2050E72
:1003CA0001D0030E7A6F0001600509E10AD8040121
:1003DA0004BD02D0C80E01D0880E046F120093EF3C
:1003EA0002F00001080E665D000E675903E266C05E
:1003FA0069F002D0080E696F69C005F46951006E90
:10040A00016A0050665F0150675B180E646F040E44
:10041A00656F69511CE000017BA307D062C0F6FF3B
:10042A0063C0F7FF0800F55005D062C0E9FF63C05A
:10043A00EAFFEF5064C0E9FF65C0EAFFEF6E000112
:10044A00622B000E6323642B65236907E2D712002F
:10045A0001C46AF000016A516625666F000E6721C1
:10046A00676F180E626F040E636F6A5111E062C003
:10047A00E9FF63C0EAFFEF5064C0E9FF65C0EAFF25
:10048A00EF6E642B000E6523622B63236A07EDD798
:10049A001200000161510BE10401080E016F100EF8
:1004AA00026F040E036F840E006F040123D004014F
:1004BA0010AF22D0000166510401165D0001675198
:1004CA000401175904E216C466F017C467F089DFFD
:1004DA000001010E606F0401080E016F100E026F19
:1004EA00040E036F800E006F0401180E066F040ECF
:1004FA00076FC80E046F10D00001020E606F04016E
:10050A00056BC80E046F0401080E016F180E026F06
:10051A00040E036FC80E006F6D9812000001606B25
:10052A000401080E016F100E026F040E036F880E8D
:10053A00006F0401046B120004011051600BE842C1
:10054A00E842E842E842E842000901E0120011519B
:10055A00080A39E0010A35E00F0A0AE0030A01E055
:10056A0012000001010E616F0001040E7A6F120081
:10057A000001010E616F0401130507E10001560E27
:10058A00626F070E636F120E13D0020E135D07E13E
:10059A000001680E626F070E636F200E09D0030E0A
:1005AA00135D0AE10001880E626F070E636F040E85
:1005BA000001666F676B02D00001616B00017B83EB
:1005CA001200F6EF02F00001010E616F00017C0ECD
:1005DA00626F000E636F00017B930001010E666F6C
:1005EA0012000001010E616F12C47CF00401125165
:1005FA0004E10001050E7A6F12000001060E7A6FFF
:10060A0016EF00F0080E6D6E6DBAFED7686A110E0D
:10061A00696E0001020E7A6F12006850040B06E040
:10062A006950040B03E06D92699468946850010B59
:10063A0004E06950010B01E027D86850100B09E06B
:10064A006950100B06E0698468986D82A08A0300DD
:10065A00A19A6850200B09E06950200B06E070A0AF
:10066A0003D093EC02F07090689A030E00017A5D51
:10067A0001E209D06850080B06E06950080B03E054
:10068A00A8EC01F068961200686A7B0E696E6E6AC1
:10069A00160E706E68A602D06896FCD76D9893EC19
:1006AA0002F000017C6B0001030E7A6F12002A0E21
:1006BA00F66E000EF76E000EF86E00010900F55096
:1006CA00706F0900F550716F03E1706701D03DD07A
:1006DA000900F5506B6F0900F5506C6F0900F55071
:1006EA006D6F09000900F550E96E0900F550EA6ED0
:1006FA00090009000900F5506E6F0900F5506F6F87
:10070A0009000900F6CF72F0F7CF73F0F8CF74F052
:10071A006BC0F6FF6CC0F7FF6DC0F8FF00016E53A7
:10072A0002E16F5307E00900F550EE6E6E07F8E23A
:10073A006F07F9D772C0F6FF73C0F7FF74C0F8FFEE
:10074A0000017007000E715BBFD712001201000290
:10075A0000000008D8040B00000000000001090294
:10076A00200001010080320904000002000000009C
:10077A00070501024000000705810240000004034A
:10078A000904C1CF7EF00F0EC1129384F16A81A4CD
:10079A0004D07EC0C1FF00EF04F0140E6F6E07ECA8
:1007AA0003F012EC03F01DEC01F0FBD7120013EE7C
:1007BA0000F023EE00F0F86A059C5CEC03F0C6EC4E
:1007CA0003F0FDD71200FFFFFFFFFFFFFFFFFFFF50
:100800003DEF0BF01200FFFF0DEF05F01200FFFFB0
:1008180099EF05F01200FFFFFFFFFFFFFFFFFFFF4B
:10082A0000007F0E936EF26AF16AF06AD09EA09A77
:10083A00880ED56EB10ECD6E0001D00EAB6F8A0E4A
:10084A00AC6FEF0EAD6FF10EAE6FAF6B040E616F52
:10085A00B66BC00E636FC70E746FC00E646FC70E9F
:10086A00756FC00E656FC70E766FC00E666FC70EC6
:10087A00776FACC0CFFFABC0CEFFAEC0D7FFADC065
:10088A00D6FFB16BB06BAF51010BF36EF346F34673
:10089A00F346F346F346F346F3467F0E8A14F31003
:1008AA008A6E040108BF0BD0250EE66E860EE66E30
:1008BA00000EE66E6DEC09F0E552E552E5521200C3
:1008CA00040108BFA4D0250EE66E860EE66E000E61
:1008DA00E66E6DEC09F0E552E552E552A00E000114
:1008EA00865D02E0000E01D0010E026E200E865DCA
:1008FA0002E0000E01D0010E021003E0010EB66FF5
:10090A0001D0B66B1F0E8615616F000EE76E861951
:10091A00E8AE02D0863503D0E750D880865502E289
:10092A00AF6B02D0010EAF6FA7C0B7F0A8C0B8F086
:10093A00B7C0B4F0B8C0B5F0B4C0B7F0B5C0B8F03D
:10094A00FF0ED880B757B857B7C0ABF0B8C0ACF0F5
:10095A00A9C0B7F0AAC0B8F0B7C0B2F0B8C0B3F037
:10096A00B2C0B7F0B3C0B8F0D880B757B857B7C05D
:10097A00ADF0B8C0AEF0010E606F110E605D33E2EB
:10098A006051E824FF0FEA6A860FE96E000EEA2238
:10099A00EFCFB7F06051E824EA6A860FE96E000EDD
:1009AA00EA22EFCFB8F0B7C0B4F0B8C0B5F0B25190
:1009BA00B45DB76FB351B559B86FFF0ED880B7574A
:1009CA00B8576051EA6A620FE96E000EEA22B7C0B0
:1009DA00EFFF6051EA6A730FE96E000EEA22B8C0AF
:1009EA00EFFF602BCAD787C0B7F088C0B8F0B7C08E
:1009FA00B4F0B8C0B5F0B4C0B7F0B5C0B8F0FF0EE7
:100A0A00D880B757B857B7C084F0B8C085F012007D
:100A1A00DACFE4FFE2CFDAFFE9CFE4FFEACFE4FF7F
:100A2A00E652F2A454D0F2940001B60503E18A8E8C
:100A3A0073D04DD0B0050CE18150800B02E08A9E44
:100A4A0001D08A8EAEC0D7FFADC0D6FFB06B64D0DE
:100A5A006151B15D02E3000E01D0010E046EB05186
:100A6A0002E0000E01D0010E04141AE08150800B3E
:100A7A0002E08A9E01D08A8EB12BB151EA6A730FC5
:100A8A00E96E000EEA22EF50D76EB151EA6A620FA0
:100A9A00E96E000EEA22EF50D66E010EB06F3CD01E
:100AAA006151B15D02E0000E01D0010E046EB05139
:100ABA0002E0000E01D0010E041408E08150800B00
:100ACA0002E08A9E01D08A8EB12B26D025D09EA024
:100ADA0023D0ACC0CFFFABC0CEFF9E900001B605BD
:100AEA0007E18A9E85C0D7FF84C0D6FFF29414D04E
:100AFA00AEC0D7FFADC0D6FFAF51010BF36EF346C0
:100B0A00F346F346F346F346F346F3467F0E8A145A
:100B1A00F3108A6EB16BB06BE552E5CFEAFFE5CF11
:100B2A00E9FFE5CFDAFF1100D8CFE4FFE0CFE4FF19
:100B3A00E46EDACFE4FFE2CFDAFFE652E552E5CF20
:100B4A00DAFFE550E5CFE0FFE5CFD8FF100004015A
:100B5A001051600BE842E842E842E842E8420009E4
:100B6A0001E055D01151070A51E00B0A4FE0070A7C
:100B7A0040E0010A2CE00B0A28E0020A26E0030AF8
:100B8A0022E0080A12E0010A0EE00F0A0AE0030A4C
:100B9A0001E03CD00001010EC46F0001040ECB6FCE
:100BAA0036D036D834D090D832D00001010EC46F76
:100BBA000001CD0EC56F000EC66F0001CC93000177
:100BCA00010EC96F24D0A8D822D0F4D820D00001B1
:100BDA00010EC46F040114510001C56FC66BCE0E1D
:100BEA00C527000EC6230001CC930001010EC96F70
:100BFA000ED00001010EC46F04011451EA6ACE0F2F
:100C0A00E96E000EEA2212C4EFFF01D000D01200F2
:100C1A00800E0401105D57E11351030A34E0010A02
:100C2A0010E0030A01E04DD00001010EC46F00017B
:100C3A00E20EC56F140EC66F120E0001C96FCA6BA1
:100C4A0040D00001010EC46F04011251F66EF76A1A
:100C5A00D890F636F736830EF626150EF7220900D7
:100C6A00F5CFC5F00A00F5CFC6F0020E0001F76A0B
:100C7A00C525F66EC651F7220900F5CFC9F00A005C
:100C8A00F5CFCAF01ED00001010EC46F0401125143
:100C9A00F66EF76AD890F636F736870EF626150EF0
:100CAA00F7220900F5CFC5F00A00F5CFC6F0C5C096
:100CBA00F6FFC6C0F7FF0800F5500001C96FCA6BFE
:100CCA0000D00001CC8312000001010EC46F0F0E88
:100CDA00E66E710EE66E0F0EE66E5CEC0AF0E552F9
:100CEA00E552E552010EE66ECE0EE66E000EE66E97
:100CFA005CEC0AF0E552E552E55212C4CDF004016B
:100D0A00125104E10001050ECB6F05D00001060E59
:100D1A00CB6F1EEC09F012000401186B196B040169
:100D2A0010511F0B020A14E0030A0EE0010A01E047
:100D3A0033D00001010EC46F040118810001CCA157
:100D4A0002D00401188328D00001010EC46F24D0F8
:100D5A000001010EC46F040114510F0B080DF3506A
:100D6A00036A000F026E040E03221451800B01E085
:100D7A00010E040DF35000010224C76F000E032078
:100D8A00C86FC7C0E9FFC8C0EAFFEF50040B03E011
:100D9A000401010E186F00D00001C4050AE1000128
:100DAA00180EC56F040EC66F0001CC930001020E27
:100DBA00C96F12000401120510E110511F0B00093E
:100DCA000CE10001010EC46F030E0401115D03E181
:100DDA000001CC8102D00001CC91040112513AE108
:100DEA0010511F0B020836E114510F0B000932E0B3
:100DFA000001010EC46F040114510F0B080DF350CA
:100E0A00036A000F026E040E03221451800B01E0E4
:100E1A00010E040DF35000010224C76F000E0320D7
:100E2A00C86F030E0401115D07E1840EC7C0E9FF14
:100E3A00C8C0EAFFEF6E0ED014AF06D0C7C0E9FFF4
:100E4A00C8C0EAFFEF6A06D0880EC7C0E9FFC8C06B
:100E5A00EAFFEF6E12006C500BE1040100513C0BEB
:100E6A00E842E8420D0802E108D801D03CD804D093
:100E7A00040E6C5C01E147D81200D9CFE6FFE1CF3E
:100E8A00D9FFE6520001C36BC46BC96BCA6BACECE9
:100E9A0005F0DF6ADF50026E036A010E025C000E83
:100EAA0003581BE20001C45101E017D0F76ADF348E
:100EBA00FE0BF736F66E8D0EF626150EF722090092
:100ECA00F5CF02F00800F5CF03F004D003C0FAFF13
:100EDA000250F96EFBDFDF2ADDD7D5D8E552E5529D
:100EEA00E7CFD9FF1200020E0001C35D0AE192D8D2
:100EFA00040100BD03D0C80E006F02D0880E006F37
:100F0A0001D007D91200040E0001CB5D0AE112C418
:100F1A006EFF6E50000803E2050ECB6F02D0030E7F
:100F2A00CB6F0001C3050AE10BD8040104BD03D04D
:100F3A00C80E046F02D0880E046F01D0EAD81200DE
:100F4A00D9CFE6FFE1CFD9FF020EE1260001080E54
:100F5A00C95D000ECA5905E2C9C0DEFFCAC0DDFF7D
:100F6A0003D0080EDE6EDD6A040104930491010EBB
:100F7A00DB500413DFCF05F4000EDB500001C95F1C
:100F8A00010EDB50CA5B180EC76F040EC86F000152
:100F9A00CCA31ED0D9CFE9FFDACFEAFFEE50ED108D
:100FAA0016E0C5C0F6FFC6C0F7FF0800F550C7C077
:100FBA00E9FFC8C0EAFFEF6E0001C72B000EC82385
:100FCA00C52BC623DF06010E01E2DB06E3D71CD0E0
:100FDA00D9CFE9FFDACFEAFFEE50ED1015E0C5C030
:100FEA00E9FFC6C0EAFFEF50C7C0E9FFC8C0EAFF81
:100FFA00EF6E0001C72B000EC823C52BC623DF06E0
:10100A00010E01E2DB06E4D7D9CFE1FFE552E7CFD3
:10101A00D9FF1200D9CFE6FFE1CFD9FF020EE126B0
:10102A00030E04010015E76E010EE7CFDBFF01C4D2
:10103A00DFFFDE500001C927DD50CA23180EC56F35
:10104A00040EC66FD9CFE9FFDACFEAFFEE50ED10F2
:10105A0014E0C5C0E9FFC6C0EAFFEF50C7C0E9FF08
:10106A00C8C0EAFFEF6EC72B000EC823C52BC623E4
:10107A00DF06010E01E2DB06E5D7D9CFE1FFE55233
:10108A00E7CFD9FF12000001C4510CE10401080E98
:10109A00016F100E026F040E036F840E006F0401BD
:1010AA00046F35D0040110AF22D00001C9510401E8
:1010BA00165D0001CA510401175904E216C4C9F0A9
:1010CA0017C4CAF03DDF0001010EC36F0401080E08
:1010DA00016F100E026F040E036F800E006F040181
:1010EA00180E066F040E076FC80E046F10D00001A9
:1010FA00020EC36F0401056BC80E046F0401080ECB
:10110A00016F180E026F040E036FC80E006F6D9800
:10111A0012000001C36B0401080E016F100E026F6A
:10112A00040E036F880E006F0401046B12000401A1
:10113A0010511F0B010801E079D0145101E076D05B
:10114A00060E115D2EE11351230A28E0010A13E06D
:10115A00030A01E024D00001020EC46F0001CD058C
:10116A0005E10001060EC56F150EC66F090E0001D6
:10117A00C96FCA6B14D00001020EC46F0001CD05FD
:10118A0005E10001610EC56F150EC66F0001CD05A0
:10119A0004E1220E0001C96FCA6B01D000D0000120
:1011AA00CC8304011051600BE842E842E842E8426D
:1011BA00E842010801E03AD011510B0A31E0080A6D
:1011CA0021E0090A19E0080A09E00B0A05E0080A01
:1011DA0001E02CD02CD82AD02BD828D00001020E1E
:1011EA00C46F0001CF0EC56F000EC66F0001CC930D
:1011FA000001010EC96F1AD00001020EC46F13C498
:10120A00CFF014D00001020EC46F0001D00EC56FDA
:10121A00000EC66F0001CC930001010EC96F06D003
:10122A000001020EC46F12C4D0F000D012001200E6
:10123A0012000001D16B1E0E716E0401250E096F9A
:10124A00200E0A6F040E0B6F880E086F0401450EFC
:10125A000E6F040E0F6F400E0C6F1200D9CFE6FF0F
:10126A00E1CFD9FFE652FC0EDB50010805E2010E80
:10127A00F36EFC0EF3CFDBFFDF6AFC0EDB50DF5CA4
:10128A0019E2DF50E76EFD0EDBCFE9FFFE0EDBCF82
:10129A00EAFFE750E926000EEA22EF50E66EDF5039
:1012AA00EA6A450FE96E040EEA22E552E750EF6E4C
:1012BA00DF2AE3D7FC0EDBCF0DF4400E04010C1736
:1012CA000C7D880E0C13E552E552E7CFD9FF1200C8
:1012DA00D9CFE6FFE1CFD9FF0001D16B040108BFE6
:1012EA0031D0FC0EDBCF02F00951D880025403E260
:1012FA00FC0E09C4DBFF0001D16BFC0EDB50D15D93
:10130A0019E2D151EA6A200FE96E040EEA22EF507F
:10131A00E66ED151E76EFD0EDBCFE9FFFE0EDBCFA5
:10132A00EAFFE750E926000EEA22E552E750EF6E9F
:10133A00D12BE3D70401250E096F400E0817087D4B
:10134A00880E08130001D15100D0E552E7CFD9FF2A
:10135A0012006DA60FD802D06DB613D80001CB05C6
:10136A0008E16DBA06D0686A696A69806988020EFE
:10137A00CB6F12006D6A696A6D860001010ECB6F30
:10138A0012006D6A696A0001CB6B1200C6EF09F0A0
:10139A000001CB5101E13AD06850040B04E06950D6
:1013AA00040B01E041D86DB231D06850010B04E062
:1013BA006950010B01E059D86850100B04E06950DC
:1013CA00100B01E024D86850400B04E06950400B30
:1013DA0001E040D86850200B04E06950200B01E07E
:1013EA003BD86850020B04E06950020B01E03BD87D
:1013FA00030E0001CB5D01E209D06850080B06E03C
:10140A006950080B03E030EC07F068961200698413
:10141A0068986D82A19AF290A08AF2860300F2B0CF
:10142A0007D8A09AF29612006D92699468941200F5
:10143A000001CCA10ED0F8DF6D840001080ED26F36
:10144A00070ED36FD207000ED35BD251D311FAE144
:10145A006D941200689C120070A003D08EEC08F004
:10146A007090689A1200689212006A6A686A9F0EFF
:10147A006B6E7B0E696E6E6A0F0EE66E710EE66E0D
:10148A000F0EE66E14D8E552E552E552160E706E4E
:10149A0068A602D06896FCD76D988EEC08F0000119
:1014AA00CC910001CD6B0001030ECB6F1200D9CF96
:1014BA00E6FFE1CFD9FFFD0EDBCFE9FFFE0EDBCF62
:1014CA00EAFFFC0EDB5004E0EE6AFC0EDB06F9D7FD
:1014DA00E552E7CFD9FF120012010002000000080E
:1014EA00D804696901000102000109022900010109
:1014FA0000803209040000020300000009210101F2
:10150A0000012222000705810301000A07050103E1
:10151A0025000A040309041003520043002D004564
:10152A00004C004500430030035000430020007483
:10153A00006F00200052004300200049006E007432
:10154A0000650072006600610063006500200056B5
:10155A000031002E0030000600FF0901A101090137
:10156A00150026FF0095017508810209011500265C
:10157A00FF00952575089102C0F414F4141D152175
:10158A001531153811FF2A0EF66E080EF76E000E89
:10159A00F86E00010900F550BE6F0900F550BF6FE3
:1015AA0003E1BE6701D03DD00900F550B96F0900CB
:1015BA00F550BA6F0900F550BB6F09000900F550E4
:1015CA00E96E0900F550EA6E090009000900F550B4
:1015DA00BC6F0900F550BD6F09000900F6CFC0F0D5
:1015EA00F7CFC1F0F8CFC2F0B9C0F6FFBAC0F7FF23
:1015FA00BBC0F8FF0001BC5302E1BD5307E009007C
:10160A00F550EE6EBC07F8E2BD07F9D7C0C0F6FF89
:10161A00C1C0F7FFC2C0F8FF0001BE07000EBF5BE2
:10162A00BFD7120016EC04F011D8060E0001CB5DEC
:10163A0002E217D8FAD7F2949E90F28A9D80F28E2F
:10164A00F28C0FD865EC04F0FCD712000F0EC11211
:10165A00140E6F6E0001CB6B0001CC6B0001CD6BD9
:10166A001200AEEC09F06FBE02D0CDEC09F0120008
:10167A0013EE00F023EE00F0F86A019CC8EC0AF0C1
:10168A0017EC0BF0FDD71200FFFFFFFFFFFFFFFF74
:020000040020DA
:020000040030CA
:0E000000240E291E0001810008800FE00F4031
:0200000400F00A
:00000001FF
